:1000000009298030A100FE30A7200130A7207530DB
:10001000A7003030BE28A101A117AF00AF08031D13
:100020001328030114280130AF020310A20CA20C04
:10003000A20CC0302205403EAF07FE30A7202F089B
:10004000A728A101A117AF00FE30A7202F08A728DD
:10005000A401AA00AB01A01124080319A0150530C2
:10006000A3002730A900103041200330A900E83058
:100070004120A90164304120A9010A3041202A0809
:100080004828A8002B08A7002A08A600D220260886
:10009000A600A3030319A011240803195228230260
:1000A000031859282608031DA011A0195928303E0D
:1000B000A7280800AD0006118611831606118611C7
:1000C0000F30860583122D08A01884283E30A70023
:1000D0008030BE203330AC0098201330A700883029
:1000E000BE2098206430BD2098206430BD2022308E
:1000F000AC009820283083200C30832006308320E9
:10010000A0142D0884282014AC00201C92288611ED
:10011000033C031C972897200530A700DC30BE2045
:10012000031408002014FE3C0319A5288615201C82
:10013000201006150F3086052C08F03986040611AC
:10014000AC0E201898283230BD202D080429A11BA0
:100150005A2883178001840AFF3E031DAA28042918
:10016000A901A800FF30A807031CA907031C042944
:100170000330A700DF30BE20B228A701E83EA6006A
:10018000A709FC30031CC728A6070318C428A60724
:100190000000A70FC4282618CD28A61CD1280000CF
:1001A000D1280800AB01AA011030AC00270DAA0D20
:1001B000AB0D2808AA022908031C290FAB0203185B
:1001C000E8282808AA0729080318290FAB070310F5
:1001D000A60DA70DAC0BD628260804291030B000B8
:1001E000A701A601AD0CAC0C031CFC282808A6072F
:1001F00029080318290FA707A70CA60CAB0CAA0CFB
:10020000B00BF2282A080429831383120313000079
:100210000800A00107309F00E03083168500FF3002
:1002200086008113831285018601203084006030AE
:10023000AA20A03084005030AA2020308400303022
:10024000A920C830B020012077305A205A205A20E7
:100250002E305A2070305A2069305A2063305A208C
:1002600062305A2061305A2073305A2069305A2047
:1002700063305A202E305A206E305A206C305A206B
:100280000B30A900B830B120012044305A2043304F
:100290005A2046305A2032305A2030305A204E30C0
:1002A0005A204C305A2041305A2020305A205A20AF
:1002B00056305A202D305A2032305A200730A900AB
:1002C000D030B12001204C305A2044305A205230D6
:1002D0005A2020305A2061305A2066305A2072301D
:1002E0005A2065305A2067305A2065305A206C30C9
:1002F0005A2065305A206E305A2086188529851F6D
:1003000083290514842905107D29012053305A20A2
:1003100069305A2067305A206E305A2061305A2096
:100320005A206C305A2020305A207A305A206F30B0
:100330005A2065305A206B305A2065305A206E3072
:100340005A20361405128316051283122A2AC30175
:100350003C03A500C90149082502031CC029E3216B
:10036000B61CBE294308A6004908A200A601A20A9D
:100370000314A60DA20BB9292608C304C90FAB2983
:10038000B2014308B100B20CB10CB20CB10CB20C0A
:10039000B10CB20CB10C0F30B2053208AD0031080F
:1003A000AC00A9010A30A800EE20B1002B08B20071
:1003B000B4014308B3000F30B3050030B405310871
:1003C0003307C3000800BA01B9010618F829013043
:1003D000B020B90A0319BA0A0B303A02031CF729F4
:1003E000031DF629B9303902031CF729A92CE52988
:1003F0009B30B0200618B614061CB610361C142A02
:10040000AD014408AC00A9011430A800EE20B100F1
:100410002B08B2003208A7003108A600A9013A3023
:10042000A800D220BD001D2A03013619013EB618CE
:10043000013A03193611031D3615C40A851401301B
:10044000A900F430B1208510A901F030A8002808D7
:10045000B1200800BB01C4013612361ABD2ABA0108
:10046000B901061C442AB90A0319BA0A0130B0209E
:10047000AF303A02031C432A031D422AC930390215
:10048000031C432AA92C312ABA01B9010618762A7D
:10049000B90A0319BA0A0A30B02036186A2A39088C
:1004A0000B3A3A04031D552A692A3908193A3A04C5
:1004B000031D5C2A8514692A39084B3A3A04031D46
:1004C000632A8510692A3908FA3A3A04031D692A11
:1004D000A92C752A11303A02031C752A031D742AAF
:1004E00095303902031C752AA92C462A41303B025B
:1004F000031C7B2AA92CBB0A3A08031D832A6530FA
:100500003902031C842A3616361CBC2AAD013B086E
:10051000AC00A9011430A800EE20B1002B08B200F5
:100520003208A7003108A600A9014130A800D22056
:10053000BD008030A1008030212053305A20693026
:100540005A2067305A206E305A2061305A205A2083
:100550006C305A2020305A2067305A2065305A209B
:1005600076305A206F305A206E305A2064305A202C
:1005700065305A206E305A202D2A361CDF2A012081
:1005800049305A206E305A2069305A2074305A202F
:1005900069305A2061305A206C305A2069305A2014
:1005A00073305A2065305A2072305A2065305A20F4
:1005B0006E305A202E305A205A205A20492B0E30A5
:1005C000BD000130A2003D080B20A101B61DF72A95
:1005D0003B3041020318EE2AC10AF62AC101173046
:1005E00045020318F52AC50AF62AC501FB2A420866
:1005F000C1004608C500051B0B2B4508031D032B36
:100600000C30C7000A2B0D304502031C0A2B0C309E
:100610004502C700102B4508C70020305A205A2039
:100620000A3047020318162B20305A208030A100D0
:10063000470828203A305A200230A40041082920D7
:10064000051B322B0C30450203182B2B61305A202E
:100650006D305A202F2B70305A206D305A201130B7
:10066000BD00342B1330BD00410803190130031DB8
:100670000301B5001E30410203190130031D0301BF
:100680003504B50001308618030135040319492BE0
:10069000812C361E7F2CE3210130C9000F30490226
:1006A0000318552BE321C90F4E2B3611B611E32148
:1006B000E321E321B61C5E2B05145F2B05101230DD
:1006C000C900143049020318682BE321C90F612BBC
:1006D000E3210730BC00A7214308C200E321361DF7
:1006E000722BB6150630BC00A7214308C600E321D3
:1006F000361D7B2BB6150630BC00A7214308BE0073
:100700000330BC00A7214308C8000530BC00A72166
:100710004308C0000830BC00A7214308BF00E32104
:10072000361D932BB615361C992BB619982B3610FF
:100730000120B6197E2C80302120A1010130480211
:10074000031DA72B4D305A2061305A20DC2B02307C
:100750004802031DB02B44305A2069305A20DC2B4C
:1007600003304802031DB92B57305A206F305A20EE
:10077000DC2B04304802031DC22B44305A206F305A
:100780005A20DC2B05304802031DCB2B56305A2053
:1007900072305A20DC2B06304802031DD42B5A300D
:1007A0005A2061305A20DC2B07304802031DDC2B15
:1007B0005A305A206F305A208030A10083302120D7
:1007C0003E08282020305A2001304002031DEF2B24
:1007D0006A305A2061305A206E305A20672C02301D
:1007E0004002031DFA2B66305A2065305A206230D1
:1007F0005A20672C03304002031D052C6D305A200F
:1008000072305A2074305A20672C04304002031D85
:10081000102C61305A2070305A2072305A20672CC8
:1008200005304002031D1B2C6D305A2065305A20C4
:1008300069305A20672C06304002031D262C6A308E
:100840005A2075305A206E305A20672C07304002EB
:10085000031D312C6A305A2075305A206C305A20D2
:10086000672C08304002031D3C2C61305A20753043
:100870005A2067305A20672C09304002031D472C4C
:1008800073305A2065305A2070305A20672C0A3055
:100890004002031D522C6F305A206B305A207430A6
:1008A0005A20672C0B304002031D5D2C6E305A20FD
:1008B0006F305A2076305A20672C0C304002031DCE
:1008C000672C64305A2065305A2063305A20051B4B
:1008D000742C20305A208030A1000230A4003F0840
:1008E000292020305A207E2C20305A2027305A20B0
:1008F0008030A1000230A4003F082920802CA92CC0
:100900002A2A851F882C05128316051283128A2C29
:100910008316051683129B30B0204108031901305D
:10092000031D0301B50001308618030135040319C6
:100930009A2C0515851585140130A900F430B120D5
:100940000511851185100130A9004A30B120C40A73
:100950004C2B012047305A2065305A205A206E30E7
:100960005A2020305A2073305A2069305A2067307C
:100970005A206E305A2061305A205A206C305A204A
:10098000203084006030AA20A03084005030AA209B
:10099000203084003030A9200618B616061CB61286
:1009A00003010618013EB61A013C031DDD2CB70AEF
:1009B0000319B80A0130B020D02C0301B61A013057
:1009C000013A0319B612031DB61603010618013EBB
:1009D000B61A013C031DF22CB70A0319B80A0130FC
:1009E000B020E52C03303802DE300319370203183B
:0609F000C02C36142A2A77
:02400E00503F21
:00000001FF
